:02000000352A9F
:1000080070082000A2007108A1007208A0008A01EF
:100018008301911E702823009D181428721015283A
:1000280072141D19192803101A280314721820288D
:1000380003182028721021287214721C30282300FB
:1000480019082100D80023009D132000E80A03198D
:10005800E90A23009D170F28230019082100D8005A
:1000680058080D3A0130031D0030F1008030F000CF
:10007800803020005F067002031D44285E081F3C84
:10008800013003180030F0007108F00403195A28F1
:1000980020305E07860001305F3D87008101013016
:1000A800E0000030E1002100911264282030200097
:1000B8005E07860001305F3D8700210058088100F7
:1000C800013020005E07F00000305F3DF10070084D
:1000D800DE007108DF009112111C93282508970093
:1000E8002408960001306A07F00000306B3DF100EB
:1000F8007008EA007108EB006B08003C031D8628B5
:100108006A08073C03189228203022008C06200039
:10011800EA01EB010130EE000030EF0011100B1D79
:10012800B528950101306607F0000030673DF10001
:100138007008E6007108E7006708003C031DA62860
:1001480066081E3C0318B428103022008C062000D4
:10015800E601E701230895000130EC000030ED00CE
:100168000B112208F0002108F1002008F200090014
:1001780023009E18C1280000BC2821006108230024
:040188009A000800D1
:0A018C0071088A0070088200080064
:100196002000F801F9011030FC00710DF80DF90D81
:1001A6007408F8027508031C750FF9020318E22893
:1001B6007408F80775080318750FF9070310F00D92
:0801C600F10DFC0BD02808002C
:1001CE00200064088600210060088100860A200055
:0C01DE006208F0006308F100C620080071
:0A01EA001D30FD00FD0BF728080092
:1001F4002100DD0105305D0203180A295D085B0753
:10020400860000305C3D870020308100DD0AFC2838
:100214005D085B07860000305C3D87008101DD03DB
:100224005D085B07DE0000305C3DDF000A30F4004F
:10023400F5015908F0005A08F100CB207808F000C5
:100244007908F1003030F00721005E0886005F086D
:100254008700700881000A30F400F5015908F000A5
:100264005A08F100CB2070082100D9007108DA0087
:1002740000307106031D402900307006031D432918
:080284004529DD0312290800E1
:10028C00BC302000E2000030E300E130E40000303C
:10029C00E500FF302100A000FF30A1000030A200DB
:1002AC000030A300FF30A400FF30A5000030A600F2
:1002BC000030A700FF30A800FF30A9000030AA00D2
:1002CC000030AB0023009E1690309D0021008C1452
:1002DC000C142000911E762923001908F0006F29B8
:0202EC00080008
:1002EE0012001E00F003031D7729F103031D772969
:0202FE000800F6
:10030000A3302100D4000130D500D930D600003010
:0C031000D700F0309E009D011D14080075
:10031C002100590884005A08850000080319A229F5
:10032C00590884005A0885000008E000E7202100E5
:0A033C00D90A0319DA0A8E29080015
:10034600833021009D055908F000F035F03570081E
:100356009D04F5209D149D1CB129AE291C08F100B1
:0C036600F0011B08F0040030F104080056
:100372002100DC01590884005A0885000008DB00CE
:100382005B08003A0319D3295B08E000E72021004B
:10039200DC0A5C085907840000305A3D85000008D9
:0603A200DB00C129080088
:1003A8002100151595141514951195120B118B1222
:0A03B8002000230895009E010800B4
:1003C200200011102508970024089600990199121F
:0E03D200EE01EF0131309800210011100800FB
:1003E00021005B0884005C0885000008F0007008AC
:1003F00003190D2A5B0884005C0885000008F000E2
:10040000590886005A08870070088100D90A031924
:10041000DA0ADB0A0319DC0AF029590886005A08AF
:06042000870081010800C5
:1004260021005C08003C031D222A5B08003C031DDA
:10043600222A5A08003C031D222A5908003C0318A8
:100446002B2A0130D9020030DA3BDB3BDC3B132A96
:0204560008009C
:100458000D302100E000E7200A302100E000E7200D
:0204680008008A
:10046A00C02378302100990023008C010C15033039
:10047A0024008C00220091019201250093012200A0
:10048A009D019D149D131D11063021008C00220030
:10049A0097179712171697111711971417148B019C
:1004AA002000910192010B138B13AE302100AC0096
:1004BA000030AD0023009F15CF309B009C011E1514
:1004CA004621A0302100D9008630DA000130DB0055
:1004DA000030DC00132206308C000C30E000E720EC
:1004EA0020302100D900A130DA000730DB000030CB
:1004FA00DC0013222000E001E101DE01DF0121001E
:10050A002C08D9002D08DA008D30DB008330DC009E
:10051A00F0212C08D9002D08DA008E21AE30AC006B
:10052A000030AD002000E601E701EC01ED01D42125
:10053A009501E1212C222000EA01EB01E801E90101
:10054A002100D80123009D011D169D179D1619082B
:10055A002100D8003930D9000030DA00B9212C2224
:10056A0028302100D9000030DA00B9212C2280215C
:10057A009E141E148B160B11200018141110210042
:10058A00911611140B178B17D001D101CE01CF018F
:10059A00210001305007F0000030513DF100700891
:1005AA00D0007108D1005008D9005108DA002C088F
:1005BA00DB002D08DC00FA202C08D9002D08DA000F
:1005CA00B9210930E000E72002302100D900A32137
:1005DA007008D2007108D3007008D9007108DA00D7
:1005EA002C08DB002D08DC00FA202C08D9002D0885
:1005FA00DA00B9210930E000E72000302000610666
:10060A00031D092B01306006031D1D2B203021001C
:10061A00D9000130DA00B9212000E001E10121000E
:10062A00D8012000DE01DF01E801E901210091166D
:10063A00003020006D06031D242B00306C06031DBC
:10064A00272B1D2BEC01ED015E082100D9002000AB
:10065A005F082100DA002C08DB002D08DC00FA20F4
:10066A002C08D9002D08DA00B921200068082100D9
:10067A00D900200069082100DA002C08DB002D08C7
:10068A00DC00FA202C08D9002D08DA00B9212C2226
:04069A00CD2A4E2BEC
:1007800052308400833085003B30F0000130F100AE
:0C0790002330860000308700772108002D
:0206A400003420
:0806A600DB340B340034003496
:1006AE004C3465346334743420344134443443342C
:1006BE003234203452344134323420340A340D343E
:0206CE000034F6
:1006D0004934543420345534413452345434203461
:1006E0005234413430342D34523441343134203496
:1006F00026342034543469346D34653472343034E3
:10070000203426342034543469346D3465347234E2
:0A071000313420340A340D34003473
:10071A004D3469346B3472346F346334203470343A
:10072A0072346F34203435342E3436343134203434
:10073A00323431342F34303437342F343234303485
:0A074A00313432340A340D34003427
:10075400313432344634313438343434303420345F
:10076400203461347634653463342034443453346F
:0C0774003234373435340A340D3400348C
:020000040001F9
:04000E00840913341A
:00000001FF
